:020000040000FA
:0A0000000000000049EF01F05ED19E
:08001800B1D19EA8FED7AD6E28
:1000200012000C6A0B6EFF0E0B260C2200D0D8A01B
:100030001200030E0A6EE60E02D8F5D70A6AFE0F0A
:10004000096EE86A0A5AD8A012000000090600D01A
:10005000F8D71450105C196E11E2196C105014C0CE
:1000600010F0146E115015C011F0156E125016C01C
:1000700012F0166E135017C013F0176E1A0E196097
:1000800074D0145272E0186A11501C6E15181B6E51
:10009000118E158E080E195E08E317C018F016C0F1
:1000A00017F015C016F0156AF5D7192607E0D89095
:1000B0001532163217321832192EF9D71BAE33D03B
:1000C0001750135E1650125A1550115A07E2D88075
:1000D000000E135612561156800E1C1A186C04E0AE
:1000E0001306000E125A115A040E196E11660DD025
:1000F00012C011F013C012F018C013F0186A080EE5
:10010000105E29E3192EF2D726D011BE08D0D89060
:100110001836133612361136102EF7D71CD018AEFB
:1001200022D0186A0FD017501326165012221550DD
:10013000112206E31132123213321832104A0DD056
:1001400018AE11D0133E0FD0123E0DD0113E0BD081
:10015000D8801390EFD7106A02D01A821068136A01
:10016000126A800E116E1CAE119E1350120010C048
:100170001CF0115013C011F0136E13361C321332E1
:100180001A6A13361C3602E31A841A7E06E11A80B4
:100190001C6A136A126A116A0BD01C2803E0D8800B
:1001A000133206D0D890133202E11A8201D01A8697
:1001B0001AB604D01AA20FD01AB407D07F0E136E4D
:1001C000FF0E126E116E106E23D0800E136E01D0D2
:1001D000136A000EF6D71AB0FBD7106A9F0E1C6088
:1001E000EBD77E0E1C64F4D79E0E1C5C07E0D89003
:1001F00013321232113210321C2AF6D71AA408D048
:10020000D880000E105611561256135613AEE0D772
:1002100010501200126A136A1B9E0AD01B9E13AE66
:1002200007D0D880000E10561156125613561B8E4A
:10023000960E1C6E135209E0080E1C2611C010F019
:1002400012C011F013C012F011D012520FE1080EBB
:100250001C5E115007E1080E1C5E105002E11350A5
:1002600010D0106A126E10C011F0106A12BE06D0C3
:10027000D8901036113612361C06F8D71BAE129ED7
:100280001C5010C013F0106E125011C012F0116EFD
:100290001200400E1A6E006A4F0EAF6EB06A240E46
:1002A000AC6E900EAB6E00010F0EC16E070EB46EF9
:1002B000C69AC00E926EE00E936EC00E946E956A52
:1002C000E80E966E6ED0F2A409D0F2941F4A202A4E
:1002D000D6CF1DF0D7CF1EF0817A11009EAA19D07B
:1002E000060EAB1412E1E2CF76F0E1CF75F0772A7B
:1002F00010EEF7F07750E126000EE222AECFE7FFD6
:1003000076C0E2FF75C0E1FF1100AE50AE50AB9871
:10031000AB8811007750785C14E0782AEACF0AF0B5
:10032000E9CF09F000EEF7F07850E926000EEA2256
:10033000EF50746E0AC0EAFF09C0E9FFD8801200CE
:1003400004D0E868746ED8A012001200776A786A48
:100350009D8A9F8AF28EF28C12009D9A00EEF7F031
:10036000010EF46EF36AF306000EF45AEE6AF450CE
:10037000F310F9E1776A786A9D8A1200F29EE0CF65
:10038000F7F3D8CFF8F3E8CFF9F3F28E0001A1929A
:10039000F29EF7C3E0FFF8C3D8FFF9C3E8FFF28E7F
:1003A0001000939A8A9A0A0E3CDE92928992929653
:1003B0008996929A899A96928D9293988A98939414
:1003C0008A9493908A90959C8C9C95988C989498FC
:1003D0008B9895948C9494928B9294968B969592FC
:1003E0008C92929489949290899092988998969000
:1003F0008D9096948D9493968A9693928A92959ED8
:100400008C9E959A8C9A949A8B9A95968C969490A9
:100410008B9094948B9495908C906C6A6B6A666ABE
:10042000656A686A676A6A6A696A00EEBFF0380ED0
:10043000EE68E82EFDD7B16BB26BB36BB46BB56BE6
:10044000B66BB76BB86BB96BBA6BBB6BBC6BBD6B88
:10045000BE6B7A6A796A7C6A7B6A7E6A7D6A806B27
:100460007F6A826B816B846B836B866B856B886B19
:10047000876B8A6B896B8C6B8B6B8E6B8D6B906BC8
:100480008F6B926B916B946B936B966B956B986B78
:10049000976B9A6B996B9C6B9B6B9E6B9D6BA06B28
:1004A0009F6BA26BA16BA46BA36BA66BA56BA86BD8
:1004B000A76BAA6BA96BAC6BAB6BAE6BAD6BB06B88
:1004C000AF6B44DF4ADFCD6AF294F28A870ED56EB5
:1004D000B16AA192A082D08EA292B10EB16E4BEC05
:1004E00011F06FEC13F02A500DEC00F0420E0DEC01
:1004F00000F0400E0DEC00F0D6CF1DF0D7CF1EF06F
:1005000009DF74C021F0C30E215C07E3FE0E215CFD
:1005100001E301D0236A89EF07F021AE29D0236AD5
:10052000820E215C05E121C023F0246825681ED0DD
:10053000920E215C05E121C023F02668276816D0C1
:10054000A20E215C05E121C023F0286829680ED0A5
:10055000B20E215C05E121C023F02A682B6806D089
:10056000C20E215C03E121C023F02C6887EF07F065
:10057000235204E189EF07F087EF07F0820E235C36
:10058000D8A4D1D0242803E121C024F0C8D021C0B0
:1005900025F04E0E245C0BE165906B90679069909E
:1005A000C269C169C069BF6989928994B5D04F0E8B
:1005B000245C0BE16592679269926B92C669C5698A
:1005C000C469C36989968990A7D0500E245C0BE159
:1005D0006594679469946B94CA69C969C869C76965
:1005E000899A899899D0510E245C0BE1659667969B
:1005F00069966B96CE69CD69CC69CB698D928D90E9
:100600008BD0520E245C0BE16598679869986B98C3
:10061000D269D169D069CF698A988D947DD0530E03
:10062000245C0BE1659A679A699A6B9AD669D569D9
:10063000D469D3698A948A966FD0540E245C0BE1F6
:10064000659C679C699C6B9CDA69D969D869D76994
:100650008A908A9261D0550E245C0BE1659E679E5C
:10066000699E6B9EDE69DD69DC69DB698C9C8C9E12
:1006700053D0560E245C0BE1669068906A906C90A3
:10068000E269E169E069DF698C988C9A45D0570E80
:10069000245C0BE1669268926A926C92E669E56965
:1006A000E469E3698B988B9A37D0580E245C0BE190
:1006B000669468946A946C94EA69E969E869E76900
:1006C0008C948C9629D0590E245C0BE16696689622
:1006D0006A966C96EE69ED69EC69EB698B928B908A
:1006E0001BD05A0E245C0BE1669868986A986C9847
:1006F000F269F169F069EF698B968B940DD05B0E0E
:10070000245C0AE1669A689A6A9A6C9AF669F569B5
:10071000F469F3698C928C90246887EF07F089EF75
:1007200007F087EF07F0920E235CD8A45FEF07F085
:10073000262804E121C026F05DEF07F021C027F054
:100740002752D8A4CCD04E0E265C0BE16590679062
:1007500069906B90C269C169C069BF6989928994C7
:10076000B9D04F0E265C0BE16592679269926B924D
:10077000C669C569C469C36989968990ABD0500EB2
:10078000265C0BE16594679469946B94CA69C969A6
:10079000C869C769899A89989DD0510E265C0BE17A
:1007A0006596679669966B96CE69CD69CC69CB697B
:1007B0008D928D908FD0520E265C0BE165986798D4
:1007C00069986B98D269D169D069CF698A988D94FC
:1007D00081D0530E265C0BE1659A679A699A6B9AF1
:1007E000D669D569D469D3698A948A9673D0540E30
:1007F000265C0BE1659C679C699C6B9CDA69D969F6
:10080000D869D7698A908A9265D0550E265C0BE12B
:10081000659E679E699E6B9EDE69DD69DC69DB69AA
:100820008C9C8C9E57D0560E265C0BE1669068908F
:100830006A906C90E269E169E069DF698C988C9A52
:1008400049D0570E265C0BE1669268926A926C92D0
:10085000E669E569E469E3698B988B9A3BD0580EA9
:10086000265C0BE1669468946A946C94EA69E96981
:10087000E869E7698C948C962DD0590E265C0BE1C3
:10088000669668966A966C96EE69ED69EC69EB6916
:100890008B928B901FD05A0E265C0BE1669868985D
:1008A0006A986C98F269F169F069EF698B968B949C
:1008B00011D05B0E265C0BE1669A689A6A9A6C9A74
:1008C000F669F569F469F3698C928C9003D0266817
:1008D00089EF07F0266887EF07F05DEF07F04E0E0F
:1008E000265C33E1658001EEF7F0D8902734E926E5
:1008F000000EEA22EECF95F0EFCF96F095511D2431
:10090000026E96511E20036E000E1F20046E000E14
:100910002020056E05C0C2F004C0C1F003C0C0F0C5
:1009200002C0BFF08982B1530DE06B8002EEF7F098
:10093000D890B135E926000EEA22EECF79F0EFCF5C
:100940007AF001D06B905BEF07F04F0E265C33E13D
:10095000658201EEF7F0D8902734E926000EEA22EE
:10096000EECF97F0EFCF98F097511D24026E98517B
:100970001E20036E000E1F20046E000E2020056E48
:1009800005C0C6F004C0C5F003C0C4F002C0C3F087
:100990008986B2530DE06B8202EEF7F0D890B23543
:1009A000E926000EEA22EECF7BF0EFCF7CF001D0FB
:1009B0006B925BEF07F0500E265C33E1658401EE2D
:1009C000F7F0D8902734E926000EEA22EECF99F00E
:1009D000EFCF9AF099511D24026E9A511E20036E9A
:1009E000000E1F20046E000E2020056E05C0CAF008
:1009F00004C0C9F003C0C8F002C0C7F0898AB3536D
:100A00000DE06B8402EEF7F0D890B335E926000EC6
:100A1000EA22EECF7DF0EFCF7EF001D06B945BEF5A
:100A200007F0510E265C33E1658601EEF7F0D890B1
:100A30002734E926000EEA22EECF9BF0EFCF9CF0A0
:100A40009B511D24026E9C511E20036E000E1F2020
:100A5000046E000E2020056E05C0CEF004C0CDF05F
:100A600003C0CCF002C0CBF08D82B4530DE06B8696
:100A700002EEF7F0D890B435E926000EEA22EECF68
:100A80007FF0EFCF80F001D06B965BEF07F0520E56
:100A9000265C32E1658801EEF7F0D8902734E9262C
:100AA000000EEA22EECF9DF0EFCF9EF09D511D2467
:100AB000026E9E511E20036E000E1F20046E000E5B
:100AC0002020056E05C0D2F004C0D1F003C0D0F0E4
:100AD00002C0CFF08A88B5530DE06B8802EEF7F0C4
:100AE000D890B535E926000EEA22EECF81F0EFCF9F
:100AF00082F001D06B98DFD1530E265C32E1658A1B
:100B000001EEF7F0D8902734E926000EEA22EECF66
:100B10009FF0EFCFA0F09F511D24026EA0511E2028
:100B2000036E000E1F20046E000E2020056E05C00F
:100B3000D6F004C0D5F003C0D4F002C0D3F08A844C
:100B4000B6530DE06B8A02EEF7F0D890B635E92681
:100B5000000EEA22EECF83F0EFCF84F001D06B9A43
:100B6000AAD1540E265C32E1658C01EEF7F0D890E4
:100B70002734E926000EEA22EECFA1F0EFCFA2F053
:100B8000A1511D24026EA2511E20036E000E1F20D3
:100B9000046E000E2020056E05C0DAF004C0D9F006
:100BA00003C0D8F002C0D7F08A80B7530DE06B8C39
:100BB00002EEF7F0D890B735E926000EEA22EECF24
:100BC00085F0EFCF86F001D06B9C75D1550E265C79
:100BD00032E1658E01EEF7F0D8902734E926000E59
:100BE000EA22EECFA3F0EFCFA4F0A3511D24026EB2
:100BF000A4511E20036E000E1F20046E000E202044
:100C0000056E05C0DEF004C0DDF003C0DCF002C0FC
:100C1000DBF08C8CB8530DE06B8E02EEF7F0D890C1
:100C2000B835E926000EEA22EECF87F0EFCF88F044
:100C300001D06B9E40D1560E265C32E1668001EEFB
:100C4000F7F0D8902734E926000EEA22EECFA5F07F
:100C5000EFCFA6F0A5511D24026EA6511E20036EF3
:100C6000000E1F20046E000E2020056E05C0E2F06D
:100C700004C0E1F003C0E0F002C0DFF08C88B9539B
:100C80000DE06C8002EEF7F0D890B935E926000E41
:100C9000EA22EECF89F0EFCF8AF001D06C900BD131
:100CA000570E265C32E1668201EEF7F0D8902734C9
:100CB000E926000EEA22EECFA7F0EFCFA8F0A75169
:100CC0001D24026EA8511E20036E000E1F20046E0C
:100CD000000E2020056E05C0E6F004C0E5F003C05C
:100CE000E4F002C0E3F08B88BA530DE06C8202EEB0
:100CF000F7F0D890BA35E926000EEA22EECF8BF055
:100D0000EFCF8CF001D06C92D6D0580E265C32E139
:100D1000668401EEF7F0D8902734E926000EEA2227
:100D2000EECFA9F0EFCFAAF0A9511D24026EAA516F
:100D30001E20036E000E1F20046E000E2020056E84
:100D400005C0EAF004C0E9F003C0E8F002C0E7F033
:100D50008C84BB530DE06C8402EEF7F0D890BB3569
:100D6000E926000EEA22EECF8DF0EFCF8EF001D013
:100D70006C94A1D0590E265C32E1668601EEF7F044
:100D8000D8902734E926000EEA22EECFABF0EFCF61
:100D9000ACF0AB511D24026EAC511E20036E000E50
:100DA0001F20046E000E2020056E05C0EEF004C06A
:100DB000EDF003C0ECF002C0EBF08B82BC530DE011
:100DC0006C8602EEF7F0D890BC35E926000EEA22D8
:100DD000EECF8FF0EFCF90F001D06C966CD05A0E22
:100DE000265C32E1668801EEF7F0D8902734E926D8
:100DF000000EEA22EECFADF0EFCFAEF0AD511D24E4
:100E0000026EAE511E20036E000E1F20046E000EF7
:100E10002020056E05C0F2F004C0F1F003C0F0F030
:100E200002C0EFF08B86BD530DE06C8802EEF7F048
:100E3000D890BD35E926000EEA22EECF91F0EFCF33
:100E400092F001D06C9837D05B0E265C32E1668A56
:100E500001EEF7F0D8902734E926000EEA22EECF13
:100E6000AFF0EFCFB0F0AF511D24026EB0511E2095
:100E7000036E000E1F20046E000E2020056E05C0BC
:100E8000F6F004C0F5F003C0F4F002C0F3F08C8279
:100E9000BE530DE06C8A02EEF7F0D890BE35E9261D
:100EA000000EEA22EECF93F0EFCF94F001D06C9ACF
:100EB00002D026682ED026682AD02BD028D0A20EA9
:100EC000235C0BE1282803E121C028F004D021C0D5
:100ED00029F0A8EC0DF01DD01AD0B20E235C0BE166
:100EE0002A2803E121C02AF004D021C02BF0A8EC6D
:100EF0000FF00FD00CD0C20E235C08E12C2804E1C7
:100F000021C02CF078EC0FF004D001D002D06EECB0
:100F10000DF00E0E735CD8B066EF0DF06F501D5CD7
:100F200070501E5871501F5872502058D8A051EF61
:100F30000DF0728E7352D8A465D06BB008D0899230
:100F400089846590C269C169C069BF6959D069A0C7
:100F500018D0658095511D24026E96511E20036E97
:100F6000000E1F20046E000E2020056E05C0C2F08A
:100F700004C0C1F003C0C0F002C0BFF08982699014
:100F80003FD067A023D0899402EEF7F0D890B13516
:100F9000E926000EEA22EECF06F0EFCF07F006506A
:100FA0001D24026E07501E20036E000E1F20046ECB
:100FB000000E2020056E05C0C2F004C0C1F003C0C1
:100FC000C0F002C0BFF0679069801AD065A018D049
:100FD000899279501D24026E7A501E20036E000EF5
:100FE0001F20046E000E2020056E05C0C2F004C054
:100FF000C1F003C0C0F002C0BFF089846780659073
:1010000050EF0DF0010E735CD8A465D06BB208D020
:10101000899689806592C669C569C469C36959D0D2
:1010200069A218D0658297511D24026E98511E2026
:10103000036E000E1F20046E000E2020056E05C0FA
:10104000C6F004C0C5F003C0C4F002C0C3F0898676
:1010500069923FD067A223D0899002EEF7F0D89032
:10106000B235E926000EEA22EECF06F0EFCF07F008
:1010700006501D24026E07501E20036E000E1F2016
:10108000046E000E2020056E05C0C6F004C0C5F039
:1010900003C0C4F002C0C3F0679269821AD065A28F
:1010A00018D089967B501D24026E7C501E20036E42
:1010B000000E1F20046E000E2020056E05C0C6F035
:1010C00004C0C5F003C0C4F002C0C3F089806782C9
:1010D000659250EF0DF0020E735CD8A465D06BB42E
:1010E00008D0899A89886594CA69C969C869C76935
:1010F00059D069A418D0658499511D24026E9A5163
:101100001E20036E000E1F20046E000E2020056EB0
:1011100005C0CAF004C0C9F003C0C8F002C0C7F0DF
:10112000898A69943FD067A423D0899802EEF7F0AA
:10113000D890B335E926000EEA22EECF06F0EFCFC5
:1011400007F006501D24026E07501E20036E000E8D
:101150001F20046E000E2020056E05C0CAF004C0DA
:10116000C9F003C0C8F002C0C7F0679469841AD000
:1011700065A418D0899A7D501D24026E7E501E20D1
:10118000036E000E1F20046E000E2020056E05C0A9
:10119000CAF004C0C9F003C0C8F002C0C7F0898813
:1011A0006784659450EF0DF0030E735CD8A465D08E
:1011B0006BB608D08D928D806596CE69CD69CC696D
:1011C000CB6959D069A618D065869B511D24026E43
:1011D0009C511E20036E000E1F20046E000E202066
:1011E000056E05C0CEF004C0CDF003C0CCF002C047
:1011F000CBF08D8269963FD067A623D08D9002EE0A
:10120000F7F0D890B435E926000EEA22EECF06F0CA
:10121000EFCF07F006501D24026E07501E20036E0C
:10122000000E1F20046E000E2020056E05C0CEF0BB
:1012300004C0CDF003C0CCF002C0CBF06796698645
:101240001AD065A618D08D927F501D24026E805151
:101250001E20036E000E1F20046E000E2020056E5F
:1012600005C0CEF004C0CDF003C0CCF002C0CBF07E
:101270008D806786659650EF0DF0040E735CD8A4E0
:1012800065D06BB808D08A988D846598D269D16989
:10129000D069CF6959D069A818D065889D511D249F
:1012A000026E9E511E20036E000E1F20046E000E63
:1012B0002020056E05C0D2F004C0D1F003C0D0F0EC
:1012C00002C0CFF08A8869983FD067A823D08D9458
:1012D00002EEF7F0D890B535E926000EEA22EECFFF
:1012E00006F0EFCF07F006501D24026E07501E20B7
:1012F000036E000E1F20046E000E2020056E05C038
:10130000D2F004C0D1F003C0D0F002C0CFF0679893
:1013100069881AD065A818D08A9881511D24026E58
:1013200082511E20036E000E1F20046E000E20202E
:10133000056E05C0D2F004C0D1F003C0D0F002C0E9
:10134000CFF08D846788659850EF0DF0050E735CC3
:10135000D8A465D06BBA08D08A948A86659AD66973
:10136000D569D469D36959D069AA18D0658A9F51C3
:101370001D24026EA0511E20036E000E1F20046E5D
:10138000000E2020056E05C0D6F004C0D5F003C0C5
:10139000D4F002C0D3F08A84699A3FD067AA23D0E0
:1013A0008A9602EEF7F0D890B635E926000EEA22CA
:1013B000EECF06F0EFCF07F006501D24026E075067
:1013C0001E20036E000E1F20046E000E2020056EEE
:1013D00005C0D6F004C0D5F003C0D4F002C0D3F0ED
:1013E000679A698A1AD065AA18D08A9483511D24F5
:1013F000026E84511E20036E000E1F20046E000E2C
:101400002020056E05C0D6F004C0D5F003C0D4F08E
:1014100002C0D3F08A86678A659A50EF0DF0060EF7
:10142000735CD8A465D06BBC08D08A908A82659C16
:10143000DA69D969D869D76959D069AC18D0658C8F
:10144000A1511D24026EA2511E20036E000E1F200A
:10145000046E000E2020056E05C0DAF004C0D9F03D
:1014600003C0D8F002C0D7F08A80699C3FD067AC37
:1014700023D08A9202EEF7F0D890B735E926000E15
:10148000EA22EECF06F0EFCF07F006501D24026EE1
:1014900007501E20036E000E1F20046E000E202039
:1014A000056E05C0DAF004C0D9F003C0D8F002C060
:1014B000D7F0679C698C1AD065AC18D08A9085519A
:1014C0001D24026E86511E20036E000E1F20046E26
:1014D000000E2020056E05C0DAF004C0D9F003C06C
:1014E000D8F002C0D7F08A82678C659C50EF0DF06F
:1014F000070E735CD8A465D06BBE08D08C9C8C8E14
:10150000659EDE69DD69DC69DB6959D069AE18D09A
:10151000658EA3511D24026EA4511E20036E000E81
:101520001F20046E000E2020056E05C0DEF004C0F2
:10153000DDF003C0DCF002C0DBF08C8C699E3FD094
:1015400067AE23D08C9E02EEF7F0D890B835E9262E
:10155000000EEA22EECF06F0EFCF07F006501D2472
:10156000026E07501E20036E000E1F20046E000E38
:101570002020056E05C0DEF004C0DDF003C0DCF005
:1015800002C0DBF0679E698E1AD065AE18D08C9CC5
:1015900087511D24026E88511E20036E000E1F20ED
:1015A000046E000E2020056E05C0DEF004C0DDF0E4
:1015B00003C0DCF002C0DBF08C8E678E659E50EFBE
:1015C0000DF0080E735CD8A464D06CB008D08C9871
:1015D0008C8A6690E269E169E069DF6959D06AA0A6
:1015E00018D06680A5511D24026EA6511E20036EE0
:1015F000000E1F20046E000E2020056E05C0E2F0D4
:1016000004C0E1F003C0E0F002C0DFF08C886A9013
:101610003FD068A023D08C9A02EEF7F0D890B9356D
:10162000E926000EEA22EECF06F0EFCF07F00650D3
:101630001D24026E07501E20036E000E1F20046E34
:10164000000E2020056E05C0E2F004C0E1F003C0EA
:10165000E0F002C0DFF068906A801AD066A018D06F
:101660008C9889511D24026E8A511E20036E000E33
:101670001F20046E000E2020056E05C0E2F004C09D
:10168000E1F003C0E0F002C0DFF08C8A6880669071
:1016900007D2090E735CD8A464D06CB208D08B98C2
:1016A0008B8A6692E669E569E469E36959D06AA2C2
:1016B00018D06682A7511D24026EA8511E20036E09
:1016C000000E1F20046E000E2020056E05C0E6F0FF
:1016D00004C0E5F003C0E4F002C0E3F08B886A9236
:1016E0003FD068A223D08B9A02EEF7F0D890BA359B
:1016F000E926000EEA22EECF06F0EFCF07F0065003
:101700001D24026E07501E20036E000E1F20046E63
:10171000000E2020056E05C0E6F004C0E5F003C011
:10172000E4F002C0E3F068926A821AD066A218D090
:101730008B988B511D24026E8C511E20036E000E5F
:101740001F20046E000E2020056E05C0E6F004C0C8
:10175000E5F003C0E4F002C0E3F08B8A6882669291
:101760009FD10A0E735CD8A464D06CB408D08C945A
:101770008C866694EA69E969E869E76959D06AA4E0
:1017800018D06684A9511D24026EAA511E20036E32
:10179000000E1F20046E000E2020056E05C0EAF02A
:1017A00004C0E9F003C0E8F002C0E7F08C846A945A
:1017B0003FD068A423D08C9602EEF7F0D890BB35CA
:1017C000E926000EEA22EECF06F0EFCF07F0065032
:1017D0001D24026E07501E20036E000E1F20046E93
:1017E000000E2020056E05C0EAF004C0E9F003C039
:1017F000E8F002C0E7F068946A841AD066A418D0B2
:101800008C948D511D24026E8E511E20036E000E8D
:101810001F20046E000E2020056E05C0EAF004C0F3
:10182000E9F003C0E8F002C0E7F08C8668846694B3
:1018300037D10B0E735CD8A464D06CB608D08B92F1
:101840008B806696EE69ED69EC69EB6959D06AA602
:1018500018D06686AB511D24026EAC511E20036E5B
:10186000000E1F20046E000E2020056E05C0EEF055
:1018700004C0EDF003C0ECF002C0EBF08B826A967E
:101880003FD068A623D08B9002EEF7F0D890BC35FD
:10189000E926000EEA22EECF06F0EFCF07F0065061
:1018A0001D24026E07501E20036E000E1F20046EC2
:1018B000000E2020056E05C0EEF004C0EDF003C060
:1018C000ECF002C0EBF068966A861AD066A618D0D3
:1018D0008B928F511D24026E90511E20036E000EBC
:1018E0001F20046E000E2020056E05C0EEF004C01F
:1018F000EDF003C0ECF002C0EBF08B8068866696DA
:10190000CFD00C0E735CD8A464D06CB808D08B9682
:101910008B846698F269F169F069EF6959D06AA819
:1019200018D06688AD511D24026EAE511E20036E84
:10193000000E1F20046E000E2020056E05C0F2F080
:1019400004C0F1F003C0F0F002C0EFF08B866A989B
:101950003FD068A823D08B9402EEF7F0D890BD3525
:10196000E926000EEA22EECF06F0EFCF07F0065090
:101970001D24026E07501E20036E000E1F20046EF1
:10198000000E2020056E05C0F2F004C0F1F003C087
:10199000F0F002C0EFF068986A881AD066A818D0F4
:1019A0008B9691511D24026E92511E20036E000EE3
:1019B0001F20046E000E2020056E05C0F2F004C04A
:1019C000F1F003C0F0F002C0EFF08B8468886698F5
:1019D00067D00D0E735CD8A463D06CBA08D08C921B
:1019E0008C80669AF669F569F469F36959D06AAA38
:1019F00018D0668AAF511D24026EB0511E20036EAE
:101A0000000E1F20046E000E2020056E05C0F6F0AB
:101A100004C0F5F003C0F4F002C0F3F08C826A9ABF
:101A20003FD068AA23D08C9002EEF7F0D890BE3554
:101A3000E926000EEA22EECF06F0EFCF07F00650BF
:101A40001D24026E07501E20036E000E1F20046E20
:101A5000000E2020056E05C0F6F004C0F5F003C0AE
:101A6000F4F002C0F3F0689A6A8A1AD066AA18D015
:101A70008C9293511D24026E94511E20036E000E11
:101A80001F20046E000E2020056E05C0F6F004C075
:101A9000F5F003C0F4F002C0F3F08C80688A669A17
:101AA0001DD820AE12D0206A1F6A1E6A1D6A666A9F
:101AB000656A686A676A6A6A696A6C6A6B6A00EE74
:101AC000BFF0380EEE68E82EFDD706D020AE04D069
:101AD000206A1F6A1E6A1D6A7CEF02F07368728EAC
:101AE000226A0E0E225C33E2D8902234E96EEA6A52
:101AF000EA36E936EA36BF0EE926000EEA22EFCFD3
:101B000002F0ECCF03F0ECCF04F0ECCF05F06F5017
:101B1000025C70500358715004587250055815E219
:101B2000D8902234E96EEA6AEA36E936EA36BF0E20
:101B3000E926000EEA22EFCF6FF0ECCF70F0ECCF89
:101B400071F0ECCF72F022C073F0222ACAE31200C7
:101B50004E0E285C1EE129C0B1F0B1530CE002EE3C
:101B6000F7F0D890B135E926000EEA22EECF79F0F1
:101B7000EFCF7AF00DD07A6A796A6B9065906790B2
:101B80006990C269C169C069BF6989948992A6DFF9
:101B9000ADD14F0E285C1EE129C0B2F0B2530CE06B
:101BA00002EEF7F0D890B235E926000EEA22EECF29
:101BB0007BF0EFCF7CF00DD07C6A7B6A6B926592F4
:101BC00067926992C669C569C469C3698990899633
:101BD00085DF8CD1500E285C1EE129C0B3F0B353D1
:101BE0000CE002EEF7F0D890B335E926000EEA22B9
:101BF000EECF7DF0EFCF7EF00DD07E6A7D6A6B94E4
:101C0000659467946994CA69C969C869C7698998FC
:101C1000899A64DF6BD1510E285C1EE129C0B4F0B3
:101C2000B4530CE002EEF7F0D890B435E926000E7C
:101C3000EA22EECF7FF0EFCF80F00DD0806B7F6A8D
:101C40006B96659667966996CE69CD69CC69CB69C6
:101C50008D908D9243DF4AD1520E285C1EE129C03F
:101C6000B5F0B5530CE002EEF7F0D890B535E926A3
:101C7000000EEA22EECF81F0EFCF82F00DD0826B22
:101C8000816B6B98659867986998D269D169D069BA
:101C9000CF698D948A9822DF29D1530E285C1EE1EA
:101CA00029C0B6F0B6530CE002EEF7F0D890B63586
:101CB000E926000EEA22EECF83F0EFCF84F00DD0BC
:101CC000846B836B6B9A659A679A699AD669D569B2
:101CD000D469D3698A968A9401DF08D1540E285CAE
:101CE0001EE129C0B7F0B7530CE002EEF7F0D89030
:101CF000B735E926000EEA22EECF85F0EFCF86F069
:101D00000DD0866B856B6B9C659C679C699CDA69C2
:101D1000D969D869D7698A928A90E0DEE7D0550EF2
:101D2000285C1EE129C0B8F0B8530CE002EEF7F0D1
:101D3000D890B835E926000EEA22EECF87F0EFCF33
:101D400088F00DD0886B876B6B9E659E679E699E41
:101D5000DE69DD69DC69DB698C9E8C9CBFDEC6D0E8
:101D6000560E285C1EE129C0B9F0B9530CE002EE12
:101D7000F7F0D890B935E926000EEA22EECF89F0C7
:101D8000EFCF8AF00DD08A6B896B6C90669068906B
:101D90006A90E269E169E069DF698C9A8C989EDE5D
:101DA000A5D0570E285C1EE129C0BAF0BA530CE04A
:101DB00002EEF7F0D890BA35E926000EEA22EECF0F
:101DC0008BF0EFCF8CF00DD08C6B8B6B6C9266929E
:101DD00068926A92E669E569E469E3698B9A8B988F
:101DE0007DDE84D0580E285C1EE129C0BBF0BB53B9
:101DF0000CE002EEF7F0D890BB35E926000EEA229F
:101E0000EECF8DF0EFCF8EF00DD08E6B8D6B6C948E
:101E1000669468946A94EA69E969E869E7698C9666
:101E20008C945CDE63D0590E285C1EE129C0BCF0A6
:101E3000BC530CE002EEF7F0D890BC35E926000E5A
:101E4000EA22EECF8FF0EFCF90F00DD0906B8F6B3A
:101E50006C96669668966A96EE69ED69EC69EB6930
:101E60008B908B923BDE42D05A0E285C1EE129C03B
:101E7000BDF0BD530CE002EEF7F0D890BD35E92679
:101E8000000EEA22EECF91F0EFCF92F00DD0926BE0
:101E9000916B6C98669868986A98F269F169F06934
:101EA000EF698B948B961ADE21D05B0E285C1EE1C5
:101EB00029C0BEF0BE530CE002EEF7F0D890BE355C
:101EC000E926000EEA22EECF93F0EFCF94F00ED089
:101ED000946B936B6C9A669A689A6A9AF669F5693C
:101EE000F469F3698C908C926EEC0DF02868120006
:101EF0002C5203E16FEC13F029D0010E2C5C03E1AE
:101F0000D2EC13F023D0020E2C5C03E1C7EC15F0E9
:101F10001DD0030E2C5C03E114EC16F017D0040E58
:101F20002C5C03E178EC16F011D0050E2C5C03E17B
:101F300065EC18F00BD0060E2C5C03E14CEC1AF0AB
:101F400005D0070E2C5C02E1B0EC1AF02C681200F0
:101F50001E0E2A5CD8A411D12B52D8A457D06C6A7B
:101F60006B6A7A6A796AB16B7C6A7B6AB26B7E6AE9
:101F70007D6AB36B806B7F6AB46B826B816BB56B70
:101F8000846B836BB66B866B856BB76B886B876B6B
:101F9000B86B8A6B896BB96B8C6B8B6BBA6B8E6B06
:101FA0008D6BBB6B906B8F6BBC6B926B916BBD6BD6
:101FB000946B936BBE6B666A656A686A676A6A6AE5
:101FC000696A00EEBFF0380EEE68E82EFDD7899200
:101FD0008996899A8D928A988A948A908C9C8C98FA
:101FE0008B988C948B928B968C92899489908998FB
:101FF0008D908D948A968A928C9E8C9A8B9A8C96D0
:102000008B908B948C906EEC0DF0B6D02BC0B1F011
:1020100002EEF7F0D8902B34E926000EEA22EECF3C
:1020200079F0EFCF7AF02BC0B2F002EEF7F0D89053
:102030002B34E926000EEA22EECF7BF0EFCF7CF0C6
:102040002BC0B3F002EEF7F0D8902B34E926000E47
:10205000EA22EECF7DF0EFCF7EF02BC0B4F002EE9F
:10206000F7F0D8902B34E926000EEA22EECF7FF06D
:10207000EFCF80F02BC0B5F002EEF7F0D8902B3404
:10208000E926000EEA22EECF81F0EFCF82F02BC0DE
:10209000B6F002EEF7F0D8902B34E926000EEA22D3
:1020A000EECF83F0EFCF84F02BC0B7F002EEF7F065
:1020B000D8902B34E926000EEA22EECF85F0EFCF40
:1020C00086F02BC0B8F002EEF7F0D8902B34E9265A
:1020D000000EEA22EECF87F0EFCF88F02BC0B9F0E8
:1020E00002EEF7F0D8902B34E926000EEA22EECF6C
:1020F00089F0EFCF8AF02BC0BAF002EEF7F0D8905B
:102100002B34E926000EEA22EECF8BF0EFCF8CF0D5
:102110002BC0BBF002EEF7F0D8902B34E926000E6E
:10212000EA22EECF8DF0EFCF8EF02BC0BCF002EEA6
:10213000F7F0D8902B34E926000EEA22EECF8FF08C
:10214000EFCF90F02BC0BDF002EEF7F0D8902B341B
:10215000E926000EEA22EECF91F0EFCF92F02BC0ED
:10216000BEF002EEF7F0D8902B34E926000EEA22FA
:10217000EECF93F0EFCF94F036D0420E2A5C04E11C
:102180002B5201E132D82FD07B0E2A5C2CE1666AFB
:10219000656A686A676A6A6A696A6C6A6B6A00EE8D
:1021A000BFF0380EEE68E82EFDD789928996899A9D
:1021B0008D928A988A948A908C9C8C988B988C9417
:1021C0008B928B968C928994899089988D908D941E
:1021D0008A968A928C9E8C9A8B9A8C968B908B94F2
:1021E0008C906EEC0DF02A681200666A656A686A67
:1021F000676A6A6A696A6C6A6B6A00EEBFF0380ED9
:10220000EE68E82EFDD789928996899A8D928A98F0
:102210008A948A908C9C8C988B988C948B928B96B9
:102220008C928994899089988D908D948A968A92BF
:102230008C9E8C9A8B9A8C968B908B948C907A6ACD
:10224000796AB16B7C6A7B6AB26B7E6A7D6AB36BBA
:10225000806B7F6AB46B826B816BB56B846B836BB5
:10226000B66B866B856BB76B886B876BB86B8A6B4D
:10227000896BB96B8C6B8B6BBA6B8E6B8D6BBB6B1D
:10228000906B8F6BBC6B926B916BBD6B946B936B14
:10229000BE6B6EEF0DF00201F869F7695C0EFA6F24
:1022A0007A0EF96F590EFC6F850EFB6F580EFE6F9C
:1022B000140EFD6F560E0301006FA90E0201FF6F91
:1022C000550E0301026F430E016F530E046FE30EB0
:1022D000036F520E066F890E056F510E086F350E93
:1022E000076F4F0E0A6FE60E096F4E0E0C6F9C0EB5
:1022F0000B6F4D0E0E6F580E0D6F4C0E106F190EAA
:102300000F6F4A0E126FDF0E116F490E146FAA0E77
:10231000136F480E166F7A0E156F470E186F4F0E1B
:10232000176F460E1A6F290E196F450E1C6F080E97
:102330001B6F430E1E6FEB0E1D6F420E206FD30EF0
:102340001F6F410E226FBF0E216F400E246FB00E23
:10235000236F3F0E266FA50E256F3E0E286F9E0E33
:10236000276F3D0E2A6F9C0E296F3C0E2C6F9E0E20
:102370002B6F3B0E2E6FA40E2D6F3A0E306FAE0EEC
:102380002F6F390E326FBC0E316F380E346FCE0E98
:10239000336F370E366FE30E356F360E386FFD0E26
:1023A000376F360E3A6F1A0E396F350E3C6F3B0E93
:1023B0003B6F340E3E6F5F0E3D6F330E406F870EE6
:1023C0003F6F320E426FB20E416F310E446FE10E1D
:1023D000436F310E466F140E456F300E486F490E35
:1023E000476F2F0E4A6F820E496F2E0E4C6FBE0E36
:1023F0004B6F2D0E4E6FFD0E4D6F2D0E506F3F0E1D
:102400004F6F2C0E526F850E516F2B0E546FCD0EE9
:10241000536F2B0E566F180E556F2A0E586F670E9E
:10242000576F290E5A6FB80E596F290E5C6F0C0E3C
:102430005B6F280E5E6F620E5D6F270E606FBC0EC5
:102440005F6F270E626F180E616F260E646F760E37
:10245000636F250E666FD80E656F250E686F3C0E94
:10246000676F240E6A6FA20E696F240E6C6F0B0EDD
:102470006B6F230E6E6F760E6D6F220E706FE40E13
:102480006F6F220E726F540E716F210E746FC60E35
:10249000736F210E766F3B0E756F200E786FB20E44
:1024A000776F200E7A6F2B0E796F1F0E7C6FA60E42
:1024B0007B6F1F0E7E6F240E7D6F1E0E806FA30E2E
:1024C0007F6F1E0E826F250E816F1D0E846FA90E09
:1024D000836F1D0E866F2E0E856F1C0E886FB60ED5
:1024E000876F1C0E8A6F3F0E896F1B0E8C6FCB0E91
:1024F0008B6F1B0E8E6F580E8D6F1A0E906FE80E3D
:102500008F6F1A0E926F790E916F1A0E946F0B0ED9
:10251000936F190E966FA00E956F190E986F360E69
:10252000976F180E9A6FCE0E996F180E9C6F680EEB
:102530009B6F180E9E6F030E9D6F170EA06FA00E5F
:102540009F6F170EA26F3F0EA16F160EA46FDF0EC6
:10255000A36F160EA66F800EA56F160EA86F240E21
:10256000A76F150EAA6FC80EA96F150EAC6F6E0E71
:10257000AB6F150EAE6F160EAD6F140EB06FBF0EB3
:10258000AF6F140EB26F690EB16F140EB46F150EEB
:10259000B36F130EB66FC20EB56F130EB86F710E18
:1025A000B76F130EBA6F210EB96F120EBC6FD20E39
:1025B000BB6F120EBE6F840EBD6F120EC06F380E51
:1025C000BF6F110EC26FED0EC16F110EC46FA30E5F
:1025D000C36F110EC66F5A0EC56F110EC86F120E63
:1025E000C76F100ECA6FCC0EC96F100ECC6F870E5E
:1025F000CB6F100ECE6F420ECD6F0F0ED06FCF6926
:10260000D26FBD0ED16F0F0ED46F7C0ED36F0F0E35
:10261000D66F3D0ED56F0E0ED86FFE0ED76F0E0E15
:10262000DA6FC00ED96F0E0EDC6F830EDB6F0E0EED
:10263000DE6F470EDD6F0E0EE06F0C0EDF6F0D0EBE
:10264000E26FD20EE16F0D0EE46F990EE36F0D0E87
:10265000E66F610EE56F0D0EE86F2A0EE76F0C0E48
:10266000EA6FF40EE96F0C0EEC6FBE0EEB6F0C0E02
:10267000EE6F8A0EED6F0C0EF06F560EEF6F0C0EB4
:10268000F26F230EF16F0B0EF46FF10EF36F0B0E62
:10269000F66FC00EF56F010E226E0001800E225CF7
:1026A0001DE202EEF7F0D8902234E926000EEA226D
:1026B000EECF06F0EFCF07F0D8900730036E06306C
:1026C000026E02EEF7F0D8902234E926000EEA22DC
:1026D00002C0EEFF03C0EFFF222ADFE31200010178
:1026E000FA6B340EF96F020E226E0001800E225C2E
:1026F00036E22204086E01EEF7F0D8900834E9269D
:10270000000EEA22EECF06F0EFCF07F006C010F081
:1027100007C011F00AEC01F013C017F012C016F058
:1027200011C015F010C014F0330E136E126E030EAC
:10273000116E840E106E29EC00F0B7EC00F0026E02
:1027400011C003F001EEF7F0D8902234E926000E14
:10275000EA2202C0EEFF03C0EFFF222AC6E3010E09
:10276000226E800E225C1DE201EEF7F0D89022343A
:10277000E926000EEA22EECF06F0EFCF07F0D89060
:102780000730036E0630026E01EEF7F0D890223467
:10279000E926000EEA2202C0EEFF03C0EFFF222A64
:1027A000E0E312000101FA6B340EF96FFC6B380E96
:1027B000FB6FFE6B3A0EFD6F0201006B3C0E0101D8
:1027C000FF6F0201026B3E0E016F046B400E036F40
:1027D000066B420E056F086B450E076F0A6B470EBE
:1027E000096F0C6B490E0B6F0E6B4C0E0D6F106B5F
:1027F0004F0E0F6F126B510E116F146B540E136F3F
:10280000166B570E156F186B5A0E176F1A6B5E0EFC
:10281000196F1C6B610E1B6F1E6B640E1D6F206B9E
:10282000680E1F6F226B6B0E216F246B6F0E236F70
:10283000266B730E256F286B770E276F2A6B7B0E26
:10284000296F2C6B800E2B6F2E6B840E2D6F306BCF
:10285000890E2F6F326B8E0E316F346B930E336F88
:10286000366B980E356F386B9D0E376F3A6BA30E33
:10287000396F3C6BA80E3B6F3E6BAE0E3D6F406BED
:10288000B40E3F6F426BBB0E416F446BC10E436F82
:10289000466BC80E456F486BCF0E476F4A6BD60E1E
:1028A000496F4C6BDE0E4B6F4E6BE60E4D6F506BEF
:1028B000EE0E4F6F526BF60E516F546B5369010E53
:1028C000566F080E556F010E586F110E576F010E9F
:1028D0005A6F1B0E596F010E5C6F250E5B6F010E58
:1028E0005E6F2F0E5D6F010E606F3A0E5F6F010E0F
:1028F000626F450E616F010E646F500E636F010EC3
:10290000666F5C0E656F010E686F680E676F010E73
:102910006A6F750E696F010E6C6F820E6B6F010E20
:102920006E6F900E6D6F010E706F9E0E6F6F010EC9
:10293000726FAC0E716F010E746FBB0E736F010E70
:10294000766FCB0E756F010E786FDB0E776F010E11
:102950007A6FEC0E796F010E7C6FFD0E7B6F020EAD
:102960007E6F0F0E7D6F020E806F210E7F6F020E45
:10297000826F340E816F020E846F480E836F020ED9
:10298000866F5D0E856F020E886F720E876F020E66
:102990008A6F880E896F020E8C6F9F0E8B6F020EEE
:1029A0008E6FB70E8D6F020E906FCF0E8F6F020E6F
:1029B000926FE80E916F030E946F020E936F030EE9
:1029C000966F1E0E956F030E986F3A0E976F030E5B
:1029D0009A6F570E996F030E9C6F750E9B6F030EC7
:1029E0009E6F940E9D6F030EA06FB40E9F6F030E2B
:1029F000A26FD50EA16F030EA46FF80EA36F040E85
:102A0000A66F1C0EA56F040EA86F410EA76F040ED3
:102A1000AA6F670EA96F040EAC6F8E0EAB6F040E1B
:102A2000AE6FB70EAD6F040EB06FE20EAF6F050E56
:102A3000B26F0E0EB16F050EB46F3B0EB36F050E85
:102A4000B66F6A0EB56F050EB86F9B0EB76F050EA9
:102A5000BA6FCE0EB96F060EBC6F020EBB6F060EBC
:102A6000BE6F380EBD6F060EC06F700EBF6F060EC4
:102A7000C26FAA0EC16F060EC46FE60EC36F070EBB
:102A8000C66F240EC56F070EC86F640EC76F070EA2
:102A9000CA6FA70EC96F070ECC6FEC0ECB6F080E76
:102AA000CE6F330ECD6F080ED06F7D0ECF6F080E38
:102AB000D26FC90ED16F090ED46F180ED36F090EE5
:102AC000D66F6A0ED56F090ED86FBF0ED76F0A0E7C
:102AD000DA6F170ED96F0A0EDC6F720EDB6F0A0EFB
:102AE000DE6FD00EDD6F0B0EE06F310EDF6F0B0E61
:102AF000E26F960EE16F0B0EE46FFE0EE36F0C0EAD
:102B0000E66F6A0EE56F0C0EE86FDA0EE76F0D0EDA
:102B1000EA6F4D0EE96F0D0EEC6FC50EEB6F0E0EEA
:102B2000EE6F410EED6F0E0EF06FC10EEF6F0F0ED8
:102B3000F26F460EF16F0F0EF46FD00EF36F100EA2
:102B4000F66F5E0EF56F010E226E0001800E225CA4
:102B50001DE201EEF7F0D8902234E926000EEA22B9
:102B6000EECF06F0EFCF07F0D8900730036E0630B7
:102B7000026E01EEF7F0D8902234E926000EEA2228
:102B800002C0EEFF03C0EFFF222ADFE312000101C3
:102B9000FA6B2F0EF96F020E226E0001800E225C7E
:102BA00020E22204086E01EEF7F0D8900834E926FE
:102BB000000EEA22EECF06F0EFCF07F0140E062447
:102BC000026E000E0720036E01EEF7F0D89022345B
:102BD000E926000EEA2202C0EEFF03C0EFFF222A20
:102BE000DCE3010E226E800E225C1DE201EEF7F0A6
:102BF000D8902234E926000EEA22EECF06F0EFCF7D
:102C000007F0D8900730036E0630026E01EEF7F041
:102C1000D8902234E926000EEA2202C0EEFF03C05B
:102C2000EFFF222AE0E312000101FA6B2E0EF96F8A
:102C3000020E226E0001800E225C37E22204086E32
:102C400001EEF7F0D8900834E926000EEA22EECF24
:102C500006F0EFCF07F006C010F007C011F00AEC45
:102C600001F013C017F012C016F011C015F010C01B
:102C700014F00A0E136ED70E126E470E116E820EEE
:102C8000106E29EC00F0B7EC00F0026E11C003F0FA
:102C900001EEF7F0D8902234E926000EEA2202C0B5
:102CA000EEFF03C0EFFF222AC5E3010E226E800E65
:102CB000225C1DE201EEF7F0D8902234E926000EE6
:102CC000EA22EECF06F0EFCF07F0D8900730036E80
:102CD0000630026E01EEF7F0D8902234E926000E9D
:102CE000EA2202C0EEFF03C0EFFF222AE0E3120057
:102CF0000101FA6B2F0EF96FFC6B320EFB6FFE6B4E
:102D0000340EFD6F0201006B350E0101FF6F0201F1
:102D1000026B370E016F046B390E036F066B3B0EAF
:102D2000056F086B3C0E076F0A6B3E0E096F0C6B4C
:102D3000400E0B6F0E6B420E0D6F106B450E0F6F3A
:102D4000126B470E116F146B490E136F166B4B0EFF
:102D5000156F186B4E0E176F1A6B500E196F1C6B98
:102D6000530E1B6F1E6B560E1D6F206B580E1F6F80
:102D7000226B5B0E216F246B5E0E236F266B610E40
:102D8000256F286B640E276F2A6B670E296F2C6BDB
:102D90006B0E2B6F2E6B6E0E2D6F306B720E2F6FB6
:102DA000326B750E316F346B790E336F366B7D0E6F
:102DB000356F386B810E376F3A6B850E396F3C6B10
:102DC000890E3B6F3E6B8E0E3D6F406B920E3F6FD8
:102DD000426B970E416F446B9C0E436F466BA10E86
:102DE000456F486BA60E476F4A6BAB0E496F4C6B35
:102DF000B10E4B6F4E6BB60E4D6F506BBC0E4F6FDE
:102E0000526BC20E516F546BC80E536F566BCF0E80
:102E1000556F586BD50E576F5A6BDC0E596F5C6B44
:102E2000E30E5B6F5E6BEA0E5D6F606BF20E5F6FC1
:102E3000626BFA0E616F010E646F020E636F010E1A
:102E4000666F0A0E656F010E686F120E676F010ED6
:102E50006A6F1B0E696F010E6C6F240E6B6F010E93
:102E60006E6F2E0E6D6F010E706F370E6F6F010E4D
:102E7000726F410E716F010E746F4C0E736F010E05
:102E8000766F560E756F010E786F610E776F010EBB
:102E90007A6F6C0E796F010E7C6F780E7B6F010E6E
:102EA0007E6F840E7D6F010E806F910E7F6F010E1D
:102EB000826F9D0E816F010E846FAB0E836F010ECA
:102EC000866FB80E856F010E886FC60E876F010E74
:102ED0008A6FD50E896F010E8C6FE40E8B6F010E19
:102EE0008E6FF30E8D6F020E906F030E8F6F020EBA
:102EF000926F140E916F020E946F250E936F020E57
:102F0000966F370E956F020E986F490E976F020EEF
:102F10009A6F5B0E996F020E9C6F6F0E9B6F020E85
:102F20009E6F830E9D6F020EA06F970E9F6F020E15
:102F3000A26FAC0EA16F020EA46FC20EA36F020EA1
:102F4000A66FD90EA56F020EA86FF00EA76F030E25
:102F5000AA6F080EA96F030EAC6F210EAB6F030EA4
:102F6000AE6F3B0EAD6F030EB06F550EAF6F030E1D
:102F7000B26F710EB16F030EB46F8D0EB36F030E8F
:102F8000B66FAA0EB56F030EB86FC80EB76F030EFB
:102F9000BA6FE70EB96F040EBC6F070EBB6F040E5D
:102FA000BE6F280EBD6F040EC06F4A0EBF6F040EB9
:102FB000C26F6D0EC16F040EC46F910EC36F040E0D
:102FC000C66FB70EC56F040EC86FDE0EC76F050E55
:102FD000CA6FC96FCC6F2F0ECB6F050ECE6F590E17
:102FE000CD6F050ED06F850ECF6F050ED26FB20E6E
:102FF000D16F050ED46FE10ED36F060ED66F110E92
:10300000D56F060ED86F430ED76F060EDA6F760EA9
:10301000D96F060EDC6FAB0EDB6F060EDE6FE10EB6
:10302000DD6F070EE06F1A0EDF6F070EE26F540EB2
:10303000E16F070EE46F900EE36F070EE66FCE0EA2
:10304000E56F080EE86F0E0EE76F080EEA6F500E80
:10305000E96F080EEC6F940EEB6F080EEE6FDB0E4F
:10306000ED6F090EF06F230EEF6F090EF26F6E0E0B
:10307000F16F090EF46FBB0EF36F0A0EF66F0B0EB5
:10308000F56F010E226E0001800E225C1DE201EE42
:10309000F7F0D8902234E926000EEA22EECF06F0AF
:1030A000EFCF07F0D8900730036E0630026E01EEC6
:1030B000F7F0D8902234E926000EEA2202C0EEFF93
:1030C00003C0EFFF222ADFE312000101FA6B2E0E8C
:1030D000F96FFC6B310EFB6FFE6B320EFD6F020160
:1030E000006B330E0101FF6F0201026B350E016FA1
:1030F000046B360E036F066B380E056F086B3A0EC5
:10310000076F0A6B3B0E096F0C6B3D0E0B6F0E6B5E
:103110003F0E0D6F106B400E0F6F126B420E116F52
:10312000146B440E136F166B460E156F186B480E1A
:10313000176F1A6B4A0E196F1C6B4C0E1B6F1E6BB0
:103140004E0E1D6F206B510E1F6F226B530E216FA1
:10315000246B550E236F266B580E256F286B5A0E65
:10316000276F2A6B5D0E296F2C6B5F0E2B6F2E6BFA
:10317000620E2D6F306B650E2F6F326B680E316FE4
:10318000346B6B0E336F366B6E0E356F386B710EA2
:10319000376F3A6B740E396F3C6B770E3B6F3E6B3B
:1031A0007B0E3D6F406B7E0E3F6F426B820E416F18
:1031B000446B860E436F466B890E456F486B8D0ED0
:1031C000476F4A6B910E496F4C6B950E4B6F4E6B70
:1031D0009A0E4D6F506B9E0E4F6F526BA20E516F39
:1031E000546BA70E536F566BAC0E556F586BB10EE8
:1031F000576F5A6BB60E596F5C6BBB0E5B6F5E6B95
:10320000C00E5D6F606BC60E5F6F626BCB0E616F41
:10321000646BD10E636F666BD70E656F686BDD0EE6
:10322000676F6A6BE30E696F6C6BEA0E6B6F6E6BA8
:10323000F10E6D6F706BF70E6F6F726BFE0E716F2C
:10324000010E746F060E736F010E766F0D0E756FA3
:10325000010E786F150E776F010E7A6F1D0E796F64
:10326000010E7C6F250E7B6F010E7E6F2D0E7D6F24
:10327000010E806F360E7F6F010E826F3E0E816FE2
:10328000010E846F470E836F010E866F510E856F9E
:10329000010E886F5A0E876F010E8A6F640E896F58
:1032A000010E8C6F6E0E8B6F010E8E6F790E8D6F0F
:1032B000010E906F830E8F6F010E926F8E0E916FC5
:1032C000010E946F9A0E936F010E966FA50E956F77
:1032D000010E986FB10E976F010E9A6FBE0E996F27
:1032E000010E9C6FCA0E9B6F010E9E6FD70E9D6FD5
:1032F000010EA06FE50E9F6F010EA26FF30EA16F7E
:10330000020EA46F010EA36F020EA66F0F0EA56F23
:10331000020EA86F1E0EA76F020EAA6F2E0EA96FC7
:10332000020EAC6F3E0EAB6F020EAE6F4E0EAD6F67
:10333000020EB06F5F0EAF6F020EB26F700EB16F04
:10334000020EB46F820EB36F020EB66F940EB56F9D
:10335000020EB86FA70EB76F020EBA6FBA0EB96F32
:10336000020EBC6FCE0EBB6F020EBE6FE20EBD6FC3
:10337000020EC06FF70EBF6F030EC26F0D0EC16F4E
:10338000030EC46F230EC36F030EC66F3A0EC56FD4
:10339000030EC86F520EC76F030ECA6F6A0EC96F55
:1033A000030ECC6F830ECB6F030ECE6F9C0ECD6FD2
:1033B000030ED06FB60ECF6F030ED26FD10ED16F4A
:1033C000030ED46FED0ED36F040ED66F0A0ED56FB9
:1033D000040ED86F270ED76F040EDA6F450ED96F23
:1033E000040EDC6F640EDB6F040EDE6F840EDD6F87
:1033F000040EE06FA50EDF6F040EE26FC70EE16FE3
:10340000040EE46FEA0EE36F050EE66F0E0EE56F35
:10341000050EE86F320EE76F050EEA6F580EE96F82
:10342000050EEC6F7F0EEB6F050EEE6FA70EED6FC6
:10343000050EF06FD00EEF6F050EF26FFB0EF16F01
:10344000060EF46F260EF36F060EF66F530EF56F31
:10345000010E226E0001800E225C1DE201EEF7F0EB
:10346000D8902234E926000EEA22EECF06F0EFCF04
:1034700007F0D8900730036E0630026E01EEF7F0C9
:10348000D8902234E926000EEA2202C0EEFF03C0E3
:10349000EFFF222ADFE312000101FA6B2D0EF96F14
:1034A000020E226E0001800E225C37E22204086EBA
:1034B00001EEF7F0D8900834E926000EEA22EECFAC
:1034C00006F0EFCF07F006C010F007C011F00AECCD
:1034D00001F013C017F012C016F011C015F010C0A3
:1034E00014F09A0E136E990E126E3B0E116E830E2F
:1034F000106E29EC00F0B7EC00F0026E11C003F082
:1035000001EEF7F0D8902234E926000EEA2202C03C
:10351000EEFF03C0EFFF222AC5E3010E226E800EEC
:10352000225C1DE201EEF7F0D8902234E926000E6D
:10353000EA22EECF06F0EFCF07F0D8900730036E07
:103540000630026E01EEF7F0D8902234E926000E24
:10355000EA2202C0EEFF03C0EFFF222AE0E31200DE
:103560000101FA6B2C0EF96FFC6B2F0EFB6FFE6BDB
:10357000310EFD6F0201006B320E0101FF6F02017F
:10358000026B340E016F046B360E036F066B380E40
:10359000056F086B390E076F0A6B3B0E096F0C6BDA
:1035A0003D0E0B6F0E6B3F0E0D6F106B420E0F6FCB
:1035B000126B440E116F146B460E136F166B480E90
:1035C000156F186B4B0E176F1A6B4D0E196F1C6B26
:1035D000500E1B6F1E6B530E1D6F206B560E1F6F10
:1035E000226B580E216F246B5B0E236F266B5F0ED0
:1035F000256F286B620E276F2A6B650E296F2C6B67
:10360000680E2B6F2E6B6C0E2D6F306B700E2F6F44
:10361000326B730E316F346B770E336F366B7B0EFC
:10362000356F386B7F0E376F3A6B840E396F3C6B9A
:10363000880E3B6F3E6B8D0E3D6F406B920E3F6F61
:10364000426B970E416F446B9C0E436F466BA10E0D
:10365000456F486BA60E476F4A6BAC0E496F4C6BBB
:10366000B20E4B6F4E6BB80E4D6F506BBE0E4F6F60
:10367000526BC40E516F546BCB0E536F566BD20E00
:10368000556F586BD90E576F5A6BE00E596F5C6BC4
:10369000E80E5B6F5E6BF00E5D6F606BF80E5F6F38
:1036A000010E626F616B646F090E636F010E666FCE
:1036B000120E656F010E686F1B0E676F010E6A6F49
:1036C000250E696F010E6C6F2F0E6B6F010E6E6F02
:1036D000390E6D6F010E706F430E6F6F010E726FBA
:1036E0004E0E716F010E746F5A0E736F010E766F6E
:1036F000650E756F010E786F710E776F010E7A6F20
:103700007E0E796F010E7C6F8B0E7B6F010E7E6FCC
:10371000980E7D6F010E806FA60E7F6F010E826F77
:10372000B40E816F010E846FC30E836F010E866F1E
:10373000D20E856F010E886FE20E876F010E8A6FC1
:10374000F20E896F020E8C6F030E8B6F020E8E6F5E
:10375000150E8D6F020E906F270E8F6F020E926FF7
:10376000390E916F020E946F4C0E936F020E966F8E
:10377000600E956F020E986F750E976F020E9A6F1E
:103780008A0E996F020E9C6FA00E9B6F020E9E6FA9
:10379000B70E9D6F020EA06FCE0E9F6F020EA26F2E
:1037A000E70EA16F030EA46FA36BA66F1A0EA56F91
:1037B000030EA86F340EA76F030EAA6F500EA96FE9
:1037C000030EAC6F6D0EAB6F030EAE6F8A0EAD6F56
:1037D000030EB06FA90EAF6F030EB26FC90EB16FBB
:1037E000030EB46FEA0EB36F040EB66F0B0EB56F17
:1037F000040EB86F2E0EB76F040EBA6F530EB96F6A
:10380000040EBC6F780EBB6F040EBE6F9F0EBD6FB3
:10381000040EC06FC70EBF6F040EC26FF00EC16FF3
:10382000050EC46F1B0EC36F050EC66F470EC56F26
:10383000050EC86F740EC76F050ECA6FA40EC96F50
:10384000050ECC6FD50ECB6F060ECE6F070ECD6F6B
:10385000060ED06F3B0ECF6F060ED26F710ED16F7A
:10386000060ED46FA90ED36F060ED66FE20ED56F7B
:10387000070ED86F1E0ED76F070EDA6F5C0ED96F6A
:10388000070EDC6F9B0EDB6F070EDE6FDD0EDD6F4C
:10389000080EE06F210EDF6F080EE26F670EE16F1A
:1038A000080EE46FB00EE36F080EE66FFB0EE56FD7
:1038B000090EE86F490EE76F090EEA6F990EE96F7E
:1038C000090EEC6FED0EEB6F0A0EEE6F420EED6F10
:1038D0000A0EF06F9B0EEF6F0A0EF26FF70EF16F8C
:1038E0000B0EF46F560EF36F0B0EF66FB80EF56FEE
:1038F000010E226E0001800E225C1DE201EEF7F047
:10390000D8902234E926000EEA22EECF06F0EFCF5F
:1039100007F0D8900730036E0630026E01EEF7F024
:10392000D8902234E926000EEA2202C0EEFF03C03E
:0A393000EFFF222ADFE31200FFD7A9
:020000040030CA
:0300010006160ED2
:020005008580F4
:060008000FC00FE00F40E5
:00000001FF
